:020000040000FA
:10000000000083018A010C28F0000308F100710848
:100010008300F00E700E0900FF308500FF3086006F
:1000200007309F0007308316810000309F000030AA
:100030008600FF308500831200308B006D20A00108
:10004000A10103017620A2000C1C24286D20A00A27
:100050002008233C03182E28A001A10A05193728DF
:10006000A20A8601051D3228A00122087E2022084E
:100070000739A400031D3E2855205328A40B42280D
:1000800028235328A40B462800235328A40B4A28CE
:1000900050235328A40B4E2891205328A40B5228F8
:1000A000C823532800308600242800308A00210805
:1000B000A300230D0E39820700226C2828226C2809
:1000C00050226C2878226C28A0226C28C8226C2828
:1000D00078236C28A0236C2808001010DE308F00D5
:1000E00018308E000C103130900008008316031376
:1000F0009B001C141A0883120313080083160313B1
:100100009A009B011C158B1355309D00AA309D0051
:100110009C148B171C11831203138C1F8D288C13B6
:10012000080000308A002008820718343C34183454
:100130005A341834993418345A3418343C34183436
:100140005A341834993418345A3418343C34183426
:100150005A341834993418345A340034FF34003483
:10016000FF340034FF340034FF340034FF340034F3
:02017000FF345A
:1004000002308A0020088207AA34AA34AA34AA3407
:10041000AA34AA34553455345534553455345534EA
:10042000AA34AA34AA34AA34AA34AA345534553486
:100430005534553455345534AA34AA34AA34AA3420
:10044000AA34AA34553455345534553455345534BA
:1004500002308A0020088207AA340034AA3400340B
:10046000AA34003455340034553400345534003443
:10047000AA340034AA340034AA3400345534003489
:100480005534003455340034AA340034AA340034CE
:10049000AA34003455340034553400345534003413
:1004A00002308A0020088207F034F034F034F0344F
:1004B000F034F0340F340F340F340F340F340F3462
:1004C000F034F034F034F034F034F0340F340F34CE
:1004D0000F340F340F340F34F034F034F034F03480
:1004E000F034F0340F340F340F340F340F340F3432
:1004F00002308A0020088207F0340034F0340034DF
:10050000F03400340F3400340F3400340F3400342E
:10051000F0340034F0340034F03400340F3400345C
:100520000F3400340F340034F0340034F03400342D
:10053000F03400340F3400340F3400340F340034FE
:1005400002308A0020088207F834F834F834F8348E
:10055000F834F8341F341F341F341F341F341F3451
:10056000F834F834F834F834F834F8341F341F34DD
:100570001F341F341F341F34F834F834F834F8347F
:10058000F834F8341F341F341F341F341F341F3421
:1005900002308A0020088207F8341834F8341834FE
:1005A000F83418341F3418341F3418341F341834F6
:1005B000F8341834F8341834F83418341F34183434
:1005C0001F3418341F341834F8341834F8341834FD
:1005D000F83418341F3418341F3418341F341834C6
:1006000003308A002008820700340034003480342C
:1006100080348034C034C034C034E034E034E0345A
:10062000F034F034F034F834F834F834FC34FC347A
:10063000FC34FE34FE34FE34FF34FF34FF34FF3428
:10064000FF34FE34FF34FE34FF34FE34FF34FE3416
:1006500003308A002008820700340034003401345B
:1006600001340134033403340334073407340734CA
:100670000F340F340F341F341F341F343F343F34D2
:100680003F347F347F347F34FF34FF34FF34FF3412
:10069000FF347F34FF347F34FF347F34FF347F34C2
:1006A00003308A002008820700340034003400340C
:1006B000003400341834183418341834183418340A
:1006C0003C343C343C343C343C343C347E347E3426
:1006D0007E347E347E347E34FF34FF34FF34FF3486
:1006E000FF347E34FF347E34FF347E34FF347E3476
:1006F00003308A0020088207FF34FF34FF34FF34C0
:10070000FF34FF340034003400340034003400344B
:10071000FF34FF34FF34FF34FF34FF34003400343F
:100720000034003400340034FF34FF34FF34FF342D
:10073000FF34FF340034003400340034003400341B
:1007400003308A0020088207FF340034FF3400346D
:10075000FF340034FF34FF34FF34FF34FF340034FF
:10076000FF340034FF340034FF340034FF34FF34EE
:10077000FF34FF34FF340034FF340034FF340034DE
:10078000FF340034FF34FF34FF34FF34FF340034CF
:1007900003308A0020088207033407340734073403
:1007A0000E340E340E341C341C341C3438343834BB
:1007B0003834703470347034E034E034C034E034B1
:1007C000E034E034703470347034383438343834D1
:1007D0001C341C341C340E340E340E3407340734ED
:084000000F0000000A000D0092
:02400E00513F20
:00000001FF
